:10000000C5288030A100FE305420013054207530C6
:10001000A9003030AC28A101A117B100FE30542056
:1000200031085428A401AC00AD01A0112408031923
:10003000A0150430A3002D0E22202D0822202C0E06
:1000400022202C080F39F63E0318073E0A3EA8006E
:10005000A3030319A011240803193128230203184C
:1000600038282808031DA011A0193828303E54282C
:100070000800A600AA008316051083120930AB0001
:1000800003104920AA0CAB0B412803144920260871
:10009000C02803184E2800000510502805145028C9
:1000A0000030A9005B30AC28211B3928AA00083099
:1000B00026190130AB00AA0C220884002508FF3A5B
:1000C0008005841780052508031880043C30AB2088
:1000D00025088004AB0B5B280314C02808302619C0
:1000E0000130AB00AA01220884002508FF3A8005F0
:1000F000841780052508800484130005FF3E261D13
:10010000AA0C2619AA0D3230AB20AB0B75282A0891
:100110000314C028A600261CC02822088400250835
:10012000FF3A8005841780050130A900F430AC2027
:10013000250880040130A900F430AC28AB01AA00E6
:10014000FF30AA07031CAB07031CC0280330A9001B
:10015000DF30AC20A028A901E83EA800A909FC30A6
:10016000031CB528A8070318B228A8070000A90F88
:10017000B2282818BB28A81CBF280000BF280800E8
:1001800083138312031300000800A0010130AB00A9
:10019000F4309F204030A10003200630A2008030C0
:1001A000A5000130A6008A20333056200630A20078
:1001B0008030A500A601A70103146E202708353E54
:1001C00084002A088000A70A2708083C031DDC28B1
:1001D0004030A10080300D20463039206130392078
:1001E0006D303920693039206C3039207930392030
:1001F00020303920433039206F30392064303920A5
:1002000065303920203039203D30392020303920E8
:100210000230A40035081320683039204030A10096
:10022000C0300D20533039206530392072303920EC
:1002300023303920203039203D30392020303920FA
:100240000230A400360813200230A400370813201F
:100250000230A400380813200230A400390813200B
:100260000230A4003A0813200230A4003B081320F7
:10027000683039204030A10094300D2043303920BF
:10028000523039204330392020303920563039203F
:10029000613039206C303920753039206530392093
:1002A000203039203D303920203039200230A40060
:1002B0003C081320683039203508A7000530270294
:1002C000031D8A294030A100D4300D20443039204C
:1002D0006530392076303920693039206330392053
:1002E00065303920203039203D3039202030392008
:1002F0005330392077303920693039207430392033
:1003000063303920683039202030392039203920B5
:10031000392039203508A700283027020319013079
:10032000031D0301B4003508A7002230270203197A
:100330000130031D030134040319CA294030A10010
:10034000D4300D20443039206530392076303920C2
:100350006930392063303920653039202030392028
:100360003D30392020303920543039206530392053
:100370006D30392070303920203039205330392009
:10038000653039206E303920733039206F30392094
:10039000723039203508A70001302702031DFA29E1
:1003A0004030A100D4300D20443039206530392050
:1003B0007630392069303920633039206530392072
:1003C000203039203D303920203039205330392039
:1003D0006530392072303920693039206130392058
:1003E0006C3039202030392023303920203039201A
:1003F000392039202730AB0010309F20CD286300F2
:02040000FF29D2
:02400E00223F4F
:00000001FF
